:0200000480007A
:100000006F00C004732F2034930F8000630AFF0336
:10001000930F90006306FF03930FB0006302FF038A
:10002000170F0080130F0FFE63040F0067000F000F
:10003000732F203463540F006F004000136E9E53E3
:10004000171F00002320CFFD6FF09FFF732540F1A5
:100050006310050073251030635805000F00F00F82
:10006000130E100073000000130E00009702000032
:10007000938282F973905230735020307350303035
:1000800073504030970200809382C2F7638C020065
:10009000739052109302B01A739022307323203061
:1000A000E39E62F873500030970200009382420191
:1000B00073901234732540F17300203093000000D8
:1000C00093A10000930E0000130E20006392D1272D
:1000D0009300100093A11000930E0000130E300047
:1000E0006398D1259300300093A17000930E100007
:1000F000130E4000639ED1239300700093A1300043
:10010000930E0000130E50006394D123930000005F
:1001100093A10080930E0000130E6000639AD1211A
:10012000B700008093A10000930E1000130E700022
:100130006390D121B700008093A10080930E10003E
:10014000130E80006396D11F9300000093A1F07FEF
:10015000930E1000130E9000639CD11DB700008019
:100160009380F0FF93A10000930E0000130EA000F7
:100170006390D11DB70000809380F0FF93A1F07FC2
:10018000930E0000130EB0006394D11BB7000080E3
:1001900093A1F07F930E1000130EC000639AD11943
:1001A000B70000809380F0FF93A10080930E0000C1
:1001B000130ED000639ED1179300000093A1F0FFAF
:1001C000930E0000130EE0006394D1179300F0FF2C
:1001D00093A11000930E1000130EF000639AD11536
:1001E0009300F0FF93A1F0FF930E0000130E0001A7
:1001F0006390D1159300B00093A0D000930E10002F
:10020000130E10016396D013130200009300F00048
:1002100093A1A00013830100130212009302200097
:10022000E31652FE930E0000130E20016312D31149
:10023000130200009300A00093A10001130000002E
:10024000138301001302120093022000E31452FEF4
:10025000930E1000130E3001631CD30D1302000027
:100260009300000193A19000130000001300000010
:10027000138301001302120093022000E31252FEC6
:10028000930E0000130E40016314D30B1302000001
:100290009300B00093A1F00013021200930220001B
:1002A000E31852FE930E1000130E50016392D10911
:1002B00013020000930010011300000093A18000BE
:1002C0001302120093022000E31652FE930E000068
:1002D000130E6001639ED105130200009300C0005D
:1002E000130000001300000093A1E00013021200AD
:1002F00093022000E31452FE930E1000130E7001BF
:100300006398D1039320F0FF930E0000130E800139
:100310006390D003B700FF009380F00F13A0F0FFAD
:10032000930E0000130E90016314D001631CC001F2
:100330000F00F00F63000E00131E1E00136E1E0050
:10034000730000000F00F00F130E10007300000088
:10035000731000C00000000000000000000000005A
:10036000000000000000000000000000000000008D
:10037000000000000000000000000000000000007D
:040380000000000079
:1010000000000000000000000000000000000000E0
:1010100000000000000000000000000000000000D0
:1010200000000000000000000000000000000000C0
:1010300000000000000000000000000000000000B0
:081040000000000000000000A8
:040000058000200057
:00000001FF
